
 Start         Length     Name                   Class
 0001:00000000 0000A52CH .text                   CODE
 0002:00000000 00000130H .data                   DATA
 0002:00000130 00000065H .bss                    BSS


Detailed map of segments

 0001:00000000 00000196 C=CODE     S=.text    G=(none)   M=System   ACBP=A9
 0001:00000198 000001EC C=CODE     S=.text    G=(none)   M=SysInit  ACBP=A9
 0001:00000384 00000130 C=CODE     S=.text    G=(none)   M=Windows  ACBP=A9
 0001:000004B4 0000000E C=CODE     S=.text    G=(none)   M=Types    ACBP=A9
 0001:000004C4 00000038 C=CODE     S=.text    G=(none)   M=Messages ACBP=A9
 0001:000004FC 0000008E C=CODE     S=.text    G=(none)   M=SysUtils ACBP=A9
 0001:0000058C 0000000E C=CODE     S=.text    G=(none)   M=SysConst ACBP=A9
 0001:0000059C 00000106 C=CODE     S=.text    G=(none)   M=Classes  ACBP=A9
 0001:000006A4 0000001E C=CODE     S=.text    G=(none)   M=ActiveX  ACBP=A9
 0001:000006C4 00000016 C=CODE     S=.text    G=(none)   M=TypInfo  ACBP=A9
 0001:000006DC 0000000E C=CODE     S=.text    G=(none)   M=Variants ACBP=A9
 0001:000006EC 0000000E C=CODE     S=.text    G=(none)   M=VarUtils ACBP=A9
 0001:000006FC 0000000E C=CODE     S=.text    G=(none)   M=RTLConsts ACBP=A9
 0001:0000070C 00000016 C=CODE     S=.text    G=(none)   M=Graphics ACBP=A9
 0001:00000724 0000000E C=CODE     S=.text    G=(none)   M=Consts   ACBP=A9
 0001:00000734 0000025E C=CODE     S=.text    G=(none)   M=Controls ACBP=A9
 0001:00000994 0000000E C=CODE     S=.text    G=(none)   M=ActnList ACBP=A9
 0001:000009A4 0000000E C=CODE     S=.text    G=(none)   M=Contnrs  ACBP=A9
 0001:000009B4 0000000E C=CODE     S=.text    G=(none)   M=Math     ACBP=A9
 0001:000009C4 00000016 C=CODE     S=.text    G=(none)   M=ImgList  ACBP=A9
 0001:000009DC 00000074 C=CODE     S=.text    G=(none)   M=CommCtrl ACBP=A9
 0001:00000A50 00000016 C=CODE     S=.text    G=(none)   M=Forms    ACBP=A9
 0001:00000A68 0000000E C=CODE     S=.text    G=(none)   M=HelpIntfs ACBP=A9
 0001:00000A78 0000000E C=CODE     S=.text    G=(none)   M=MultiMon ACBP=A9
 0001:00000A88 00000038 C=CODE     S=.text    G=(none)   M=Imm      ACBP=A9
 0001:00000AC0 0000000E C=CODE     S=.text    G=(none)   M=Menus    ACBP=A9
 0001:00000AD0 0000000E C=CODE     S=.text    G=(none)   M=Themes   ACBP=A9
 0001:00000AE0 0000000E C=CODE     S=.text    G=(none)   M=UxTheme  ACBP=A9
 0001:00000AF0 0000000E C=CODE     S=.text    G=(none)   M=SyncObjs ACBP=A9
 0001:00000B00 0000046E C=CODE     S=.text    G=(none)   M=ComCtrls ACBP=A9
 0001:00000F70 000000EC C=CODE     S=.text    G=(none)   M=ShlObj   ACBP=A9
 0001:0000105C 00000038 C=CODE     S=.text    G=(none)   M=UrlMon   ACBP=A9
 0001:00001094 00000038 C=CODE     S=.text    G=(none)   M=WinInet  ACBP=A9
 0001:000010CC 00000038 C=CODE     S=.text    G=(none)   M=RegStr   ACBP=A9
 0001:00001104 00000050 C=CODE     S=.text    G=(none)   M=ShellAPI ACBP=A9
 0001:00001154 00000016 C=CODE     S=.text    G=(none)   M=ListActns ACBP=A9
 0001:0000116C 0000000E C=CODE     S=.text    G=(none)   M=ExtCtrls ACBP=A9
 0001:0000117C 0000009E C=CODE     S=.text    G=(none)   M=StdCtrls ACBP=A9
 0001:0000121C 0000000E C=CODE     S=.text    G=(none)   M=WinHelpViewer ACBP=A9
 0001:0000122C 0000000E C=CODE     S=.text    G=(none)   M=StdActns ACBP=A9
 0001:0000123C 0000000E C=CODE     S=.text    G=(none)   M=Dialogs  ACBP=A9
 0001:0000124C 0000000E C=CODE     S=.text    G=(none)   M=Printers ACBP=A9
 0001:0000125C 00000038 C=CODE     S=.text    G=(none)   M=WinSpool ACBP=A9
 0001:00001294 00000038 C=CODE     S=.text    G=(none)   M=CommDlg  ACBP=A9
 0001:000012CC 00000038 C=CODE     S=.text    G=(none)   M=Dlgs     ACBP=A9
 0001:00001304 0000000E C=CODE     S=.text    G=(none)   M=StrUtils ACBP=A9
 0001:00001314 0000000E C=CODE     S=.text    G=(none)   M=Clipbrd  ACBP=A9
 0001:00001324 0000000E C=CODE     S=.text    G=(none)   M=FlatSB   ACBP=A9
 0001:00001334 0000000E C=CODE     S=.text    G=(none)   M=ToolWin  ACBP=A9
 0001:00001344 00000038 C=CODE     S=.text    G=(none)   M=RichEdit ACBP=A9
 0001:0000137C 0000000E C=CODE     S=.text    G=(none)   M=ExtActns ACBP=A9
 0001:0000138C 0000000E C=CODE     S=.text    G=(none)   M=Registry ACBP=A9
 0001:0000139C 0000000E C=CODE     S=.text    G=(none)   M=IniFiles ACBP=A9
 0001:000013AC 0000000E C=CODE     S=.text    G=(none)   M=ExtDlgs  ACBP=A9
 0001:000013BC 0000000E C=CODE     S=.text    G=(none)   M=Buttons  ACBP=A9
 0001:000013CC 0000000E C=CODE     S=.text    G=(none)   M=Mapi     ACBP=A9
 0001:000013DC 0000000E C=CODE     S=.text    G=(none)   M=ComStrs  ACBP=A9
 0001:000013EC 00000080 C=CODE     S=.text    G=(none)   M=ShellConsts ACBP=A9
 0001:0000146C 00000016 C=CODE     S=.text    G=(none)   M=ComObj   ACBP=A9
 0001:00001484 0000000E C=CODE     S=.text    G=(none)   M=ComConst ACBP=A9
 0001:00001494 00008E78 C=CODE     S=.text    G=(none)   M=ShellCtrls ACBP=A9
 0001:0000A30C 0000021D C=CODE     S=.text    G=(none)   M=vclshlctrls ACBP=A9
 0002:00000000 0000002C C=DATA     S=.data    G=DGROUP   M=SysInit  ACBP=A9
 0002:0000002C 00000050 C=DATA     S=.data    G=DGROUP   M=ShlObj   ACBP=A9
 0002:0000007C 00000072 C=DATA     S=.data    G=DGROUP   M=ShellCtrls ACBP=A9
 0002:00001000 00000010 C=BSS      S=.bss     G=DGROUP   M=SysInit  ACBP=A9
 0002:00001010 00000004 C=BSS      S=.bss     G=DGROUP   M=Windows  ACBP=A9
 0002:00001014 00000004 C=BSS      S=.bss     G=DGROUP   M=Messages ACBP=A9
 0002:00001018 00000004 C=BSS      S=.bss     G=DGROUP   M=CommCtrl ACBP=A9
 0002:0000101C 00000004 C=BSS      S=.bss     G=DGROUP   M=Imm      ACBP=A9
 0002:00001020 00000004 C=BSS      S=.bss     G=DGROUP   M=ShlObj   ACBP=A9
 0002:00001024 00000004 C=BSS      S=.bss     G=DGROUP   M=UrlMon   ACBP=A9
 0002:00001028 00000004 C=BSS      S=.bss     G=DGROUP   M=WinInet  ACBP=A9
 0002:0000102C 00000004 C=BSS      S=.bss     G=DGROUP   M=RegStr   ACBP=A9
 0002:00001030 00000004 C=BSS      S=.bss     G=DGROUP   M=ShellAPI ACBP=A9
 0002:00001034 00000004 C=BSS      S=.bss     G=DGROUP   M=WinSpool ACBP=A9
 0002:00001038 00000004 C=BSS      S=.bss     G=DGROUP   M=CommDlg  ACBP=A9
 0002:0000103C 00000004 C=BSS      S=.bss     G=DGROUP   M=Dlgs     ACBP=A9
 0002:00001040 00000004 C=BSS      S=.bss     G=DGROUP   M=RichEdit ACBP=A9
 0002:00001044 00000004 C=BSS      S=.bss     G=DGROUP   M=ShellConsts ACBP=A9
 0002:00001048 0000001C C=BSS      S=.bss     G=DGROUP   M=ShellCtrls ACBP=A9


  Address         Publics by Name

 0002:00001014       .1
 0002:00001018       .1
 0002:0000101C       .1
 0002:00001020       .1
 0002:00001024       .1
 0002:00001008       .1
 0002:00001028       .1
 0002:0000102C       .1
 0002:00001030       .1
 0002:00001038       .1
 0002:0000103C       .1
 0002:00001040       .1
 0002:00001044       .1
 0002:00001048       .21
 0002:00001010       .3
 0002:00001034       .3
 0001:0000A504       @GetPackageInfoTable
 0001:000002D0       @InitPkg
 0001:00000334       @PackageLoad
 0001:0000A50C       @PackageLoad
 0001:00000340       @PackageUnload
 0001:0000A518       @PackageUnload
 0001:00009A24       AddColumn
 0001:00009B3C       AddDefaultColumn
 0001:00009BA4       AddDefaultColumns
 0001:00005774       AddDetail
 0001:000001D0       AllocTlsBuffer
 0001:000055DC       CalcFileSize
 0001:00005634       CalcModifiedDate
 0001:0000044C       ClientToScreen
 0001:00000384       CloseHandle
 0002:000000D8       cmvProperties
 0001:00009998       ColumnIsUnique
 0001:00008188       ComboSortFunc
 0001:00000A48       CommCtrl
 0001:000012C4       CommDlg
 0002:000000E8       CompareFolder
 0001:00004124       ConcatPIDLs
 0001:00000474       CopyMemory
 0001:000040F8       CopyPIDL
 0001:00004304       CreateDesktopFolder
 0001:00000394       CreateMutex
 0001:0000402C       CreatePIDL
 0001:000041F8       CreatePIDLList
 0001:00000454       CreatePopupMenu
 0001:00005050       CreateRootFolder
 0001:00004FC8       CreateRootFromPIDL
 0002:0000104C       CS
 0001:000056A0       DefaultDetailColumn
 0001:000003B4       DeleteCriticalSection
 0002:000000E4       DesktopFolder
 0001:000043DC       DesktopPIDL
 0001:000042F4       DesktopShellFolder
 0001:0000045C       DestroyMenu
 0001:00004234       DestroyPIDLList
 0001:00004180       DisposePIDL
 0001:000012FC       Dlgs
 0001:00004C9C       DoContextMenuVerb
 0001:000003BC       EnterCriticalSection
 0001:0000027C       ExitProcessTLS
 0001:00000254       ExitThreadTLS
 0001:000003C4       FileTimeToDosDateTime
 0001:000003CC       FileTimeToLocalFileTime
 0001:0000034C       Finalization
 0001:00001294       Finalization
 0001:0000A284       Finalization
 0001:00000A18       Finalization
 0001:00001344       Finalization
 0001:0000125C       Finalization
 0001:0000111C       Finalization
 0001:000010CC       Finalization
 0001:00001024       Finalization
 0001:00001094       Finalization
 0001:00001434       Finalization
 0001:0000105C       Finalization
 0001:000012CC       Finalization
 0001:000004C4       Finalization
 0001:0000047C       Finalization
 0001:00000A88       Finalization
 0001:000003D4       FindClose
 0001:000003DC       FindCloseChangeNotification
 0001:000003E4       FindFirstChangeNotification
 0001:000003EC       FindFirstFile
 0001:000003F4       FindNextChangeNotification
 0001:00000198       FreeLibrary
 0001:00004454       GetCaps
 0001:000043F8       GetCSIDLType
 0001:000003FC       GetCurrentDirectory
 0001:00005518       GetDetailsOf
 0001:00004928       GetDisplayName
 0001:000046D8       GetHasSubFolders
 0001:00004740       GetHasSubItems
 0001:00004670       GetIsFolder
 0001:00004E28       GetIShellDetails
 0001:00004D58       GetIShellFolder
 0001:00004EF8       GetIShellFolder2
 0001:000040BC       GetItemCount
 0001:00000404       GetLastError
 0001:000040D4       GetPIDLSize
 0001:0000454C       GetProperties
 0001:00004414       GetShellImage
 0001:000001DC       GetTlsSize
 0002:00001004       HInstance
 0002:000000DC       ICM
 0002:000000E0       ICM2
 0002:0000002C       IID_IContextMenu
 0002:0000004C       IID_IContextMenu2
 0002:0000006C       IID_IShellDetails
 0002:0000003C       IID_IShellFolder
 0002:0000005C       IID_IShellFolder2
 0001:000009DC       ImageList_GetIconSize
 0001:00000AB8       Imm
 0001:0000040C       InitializeCriticalSection
 0001:000002A0       InitializeModule
 0001:00000228       InitProcessTLS
 0001:000001E4       InitThreadTLS
 0001:00008718       InsertItemObject
 0001:00004A38       InvokeContextMenu
 0001:0000440C       IsElement
 0001:00000414       LeaveCriticalSection
 0001:000080D4       ListSortFunc
 0001:00000A00       ListView_EditLabel
 0001:000009E4       ListView_RedrawItems
 0001:000001A0       LocalAlloc
 0001:000001A8       LocalFree
 0001:00000444       lstrlen
 0001:000004F4       Messages
 0002:00000004       Module
 0002:00001000       ModuleIsLib
 0002:00001001       ModuleIsPackage
 0001:00004090       NextPIDL
 0002:0000007C       nFolder
 0001:00004268       NoFolderDetails
 0001:00005FC8       NotifyOptionFlags
 0001:00005E10       NotifyOptionFlags
 0001:00004A10       ObjectFlags
 0002:000000EC       R
 0001:000010FC       RegStr
 0001:000041D0       RelativeFromAbsolute
 0001:0000041C       ReleaseMutex
 0001:00001374       RichEdit
 0001:00004380       SamePIDL
 0001:00000464       SendMessage
 0001:00000424       SetCurrentDirectory
 0001:0000042C       SetErrorMode
 0001:0000114C       ShellAPI
 0001:00001464       ShellConsts
 0001:0000A2EC       ShellCtrls
 0001:0000110C       ShellExecute
 0001:00001114       ShellExecuteEx
 0001:0000100C       SHGetDesktopFolder
 0001:00001104       SHGetFileInfo
 0001:00001014       SHGetMalloc
 0001:0000101C       SHGetSpecialFolderLocation
 0001:00001054       ShlObj
 0001:0000409C       StripLastID
 0001:00004810       StrRetToString
 0001:0000037C       SysInit
 0001:00005E64       TCustomShellChangeNotifier.Change
 0001:00005EA0       TCustomShellChangeNotifier.Create
 0001:00005F08       TCustomShellChangeNotifier.Destroy
 0001:00005F78       TCustomShellChangeNotifier.SetFilters
 0001:00005F8C       TCustomShellChangeNotifier.SetOnChange
 0001:00005F50       TCustomShellChangeNotifier.SetRoot
 0001:00005FBC       TCustomShellChangeNotifier.SetWatchSubTree
 0001:0000601C       TCustomShellChangeNotifier.Start
 0001:000081B4       TCustomShellComboBox.AddItems
 0001:00008A7C       TCustomShellComboBox.Change
 0001:00007C54       TCustomShellComboBox.ClearItems
 0001:00008B50       TCustomShellComboBox.Click
 0001:00007B80       TCustomShellComboBox.Create
 0001:00007D00       TCustomShellComboBox.CreateRoot
 0001:00007E3C       TCustomShellComboBox.CreateWnd
 0001:00008A34       TCustomShellComboBox.Destroy
 0001:00007E90       TCustomShellComboBox.DestroyWnd
 0001:00008038       TCustomShellComboBox.GetFolder
 0001:000085D4       TCustomShellComboBox.GetPath
 0001:00008968       TCustomShellComboBox.GetShellImageIndex
 0001:00008490       TCustomShellComboBox.IndexFromID
 0001:000083D0       TCustomShellComboBox.Init
 0001:00008070       TCustomShellComboBox.InitItem
 0001:00008A68       TCustomShellComboBox.Loaded
 0001:00007FE4       TCustomShellComboBox.Notification
 0001:0000854C       TCustomShellComboBox.RootChanged
 0001:00007F94       TCustomShellComboBox.SetListView
 0001:00007EA4       TCustomShellComboBox.SetObjectTypes
 0001:0000861C       TCustomShellComboBox.SetPath
 0001:000087B0       TCustomShellComboBox.SetPathFromID
 0001:0000850C       TCustomShellComboBox.SetRoot
 0001:00007F44       TCustomShellComboBox.SetTreeView
 0001:00008984       TCustomShellComboBox.SetUseShellImages
 0001:00007EB8       TCustomShellComboBox.TreeUpdate
 0001:0000993C       TCustomShellListView.Back
 0001:00008D48       TCustomShellListView.ClearItems
 0001:00008DA0       TCustomShellListView.CommandCompleted
 0001:00008BF4       TCustomShellListView.Create
 0001:0000A1A8       TCustomShellListView.CreateRoot
 0001:00008FB0       TCustomShellListView.CreateWnd
 0001:00009378       TCustomShellListView.DblClick
 0001:00008D10       TCustomShellListView.Destroy
 0001:00009020       TCustomShellListView.DestroyWnd
 0001:000098E8       TCustomShellListView.DoContextPopup
 0001:00009474       TCustomShellListView.Edit
 0001:00009448       TCustomShellListView.EditText
 0001:00009C7C       TCustomShellListView.EnumColumns
 0001:00008E68       TCustomShellListView.ExecuteCommand
 0001:000097B0       TCustomShellListView.GetFolder
 0001:00009E8C       TCustomShellListView.KeyDown
 0001:000098B8       TCustomShellListView.Loaded
 0001:00009338       TCustomShellListView.Notification
 0001:00009674       TCustomShellListView.OwnerDataFetch
 0001:000097C8       TCustomShellListView.OwnerDataFind
 0001:000090E4       TCustomShellListView.Populate
 0001:0000A08C       TCustomShellListView.Refresh
 0001:00009050       TCustomShellListView.RootChanged
 0001:00009644       TCustomShellListView.SelectedFolder
 0001:00009514       TCustomShellListView.SetAutoRefresh
 0001:00009FB4       TCustomShellListView.SetComboBox
 0001:00009034       TCustomShellListView.SetObjectTypes
 0001:0000A154       TCustomShellListView.SetPathFromID
 0001:000095F4       TCustomShellListView.SetRoot
 0001:00009898       TCustomShellListView.SetSorted
 0001:00009F64       TCustomShellListView.SetTreeView
 0001:00009F40       TCustomShellListView.SetViewStyle
 0001:0000A1CC       TCustomShellListView.SynchPaths
 0001:0000A004       TCustomShellListView.TreeUpdate
 0001:0000A03C       TCustomShellListView.WndProc
 0001:000073C4       TCustomShellTreeView.CanChange
 0001:00006C7C       TCustomShellTreeView.CanExpand
 0001:0000637C       TCustomShellTreeView.ClearItems
 0001:00006484       TCustomShellTreeView.CommandCompleted
 0001:0000626C       TCustomShellTreeView.Create
 0001:00006A6C       TCustomShellTreeView.CreateRoot
 0001:00006428       TCustomShellTreeView.CreateWnd
 0001:00006F1C       TCustomShellTreeView.Delete
 0001:00006470       TCustomShellTreeView.DestroyWnd
 0001:00007984       TCustomShellTreeView.DoContextPopup
 0001:00006D9C       TCustomShellTreeView.Edit
 0001:000065C0       TCustomShellTreeView.ExecuteCommand
 0001:00006FD4       TCustomShellTreeView.FolderExists
 0001:000074DC       TCustomShellTreeView.GetFolder
 0001:00007800       TCustomShellTreeView.GetImageIndex
 0001:00007518       TCustomShellTreeView.GetPath
 0001:00007810       TCustomShellTreeView.GetSelectedIndex
 0001:00006770       TCustomShellTreeView.InitNode
 0001:00007970       TCustomShellTreeView.Loaded
 0001:00006E4C       TCustomShellTreeView.MouseUp
 0001:00006EAC       TCustomShellTreeView.NodeFromAbsoluteID
 0001:00006E68       TCustomShellTreeView.NodeFromRelativeID
 0001:00007384       TCustomShellTreeView.Notification
 0001:000068E0       TCustomShellTreeView.PopulateNode
 0001:00007088       TCustomShellTreeView.Refresh
 0001:00007068       TCustomShellTreeView.RefreshEvent
 0001:00006F48       TCustomShellTreeView.RootChanged
 0001:000074F8       TCustomShellTreeView.SelectedFolder
 0001:00007A74       TCustomShellTreeView.SetAutoRefresh
 0001:000079D4       TCustomShellTreeView.SetComboBox
 0001:00007A24       TCustomShellTreeView.SetListView
 0001:00006A58       TCustomShellTreeView.SetObjectTypes
 0001:00007544       TCustomShellTreeView.SetPath
 0001:00007640       TCustomShellTreeView.SetPathFromID
 0001:000077C0       TCustomShellTreeView.SetRoot
 0001:00007920       TCustomShellTreeView.SetUseShellImages
 0001:00007968       TCustomShellTreeView.WMDestroy
 0001:00007820       TCustomShellTreeView.WndProc
 0001:000001B0       TlsAlloc
 0002:0000100C       tlsBuffer
 0001:000001B8       TlsFree
 0001:000001C0       TlsGetValue
 0002:00000000       TlsIndex
 0002:FFBF4000       TlsLast
 0002:0000001C       TlsProc
 0001:000001C8       TlsSetValue
 0001:0000046C       TrackPopupMenu
 0001:00006708       TreeSortFunc
 0001:00006080       TShellChangeThread.Create
 0001:000060EC       TShellChangeThread.Destroy
 0001:00006128       TShellChangeThread.Execute
 0001:000061F0       TShellChangeThread.SetDirectoryOptions
 0001:00005AF8       TShellFolder.Capabilities
 0001:000051C4       TShellFolder.Create
 0001:00005330       TShellFolder.Destroy
 0001:00005C40       TShellFolder.DisplayName
 0001:00005DC4       TShellFolder.ExecuteDefault
 0001:00005380       TShellFolder.GetDetailInterface
 0001:0000599C       TShellFolder.GetDetails
 0001:00005468       TShellFolder.GetShellDetails
 0001:000054C0       TShellFolder.GetShellFolder2
 0001:00005DB8       TShellFolder.ImageIndex
 0001:00005B9C       TShellFolder.IsFolder
 0001:00005810       TShellFolder.LoadColumnDetails
 0001:00005A78       TShellFolder.ParentShellFolder
 0001:00005BEC       TShellFolder.PathName
 0001:00005AA4       TShellFolder.Properties
 0001:00005CA8       TShellFolder.Rename
 0001:00005A40       TShellFolder.SetDetails
 0001:00005B4C       TShellFolder.SubFolders
 0001:000002AC       UninitializeModule
 0001:0000108C       UrlMon
 0001:0000A524       vclshlctrls
 0001:00000434       WaitForMultipleObjects
 0001:0000043C       WaitForSingleObject
 0001:000004AC       Windows
 0001:000010C4       WinInet
 0001:0000128C       WinSpool
 0001:0000038C       _CreateMutex


  Address         Publics by Value

 0002:FFBF4000       TlsLast
 0001:00000198       FreeLibrary
 0001:000001A0       LocalAlloc
 0001:000001A8       LocalFree
 0001:000001B0       TlsAlloc
 0001:000001B8       TlsFree
 0001:000001C0       TlsGetValue
 0001:000001C8       TlsSetValue
 0001:000001D0       AllocTlsBuffer
 0001:000001DC       GetTlsSize
 0001:000001E4       InitThreadTLS
 0001:00000228       InitProcessTLS
 0001:00000254       ExitThreadTLS
 0001:0000027C       ExitProcessTLS
 0001:000002A0       InitializeModule
 0001:000002AC       UninitializeModule
 0001:000002D0       @InitPkg
 0001:00000334       @PackageLoad
 0001:00000340       @PackageUnload
 0001:0000034C       Finalization
 0001:0000037C       SysInit
 0001:00000384       CloseHandle
 0001:0000038C       _CreateMutex
 0001:00000394       CreateMutex
 0001:000003B4       DeleteCriticalSection
 0001:000003BC       EnterCriticalSection
 0001:000003C4       FileTimeToDosDateTime
 0001:000003CC       FileTimeToLocalFileTime
 0001:000003D4       FindClose
 0001:000003DC       FindCloseChangeNotification
 0001:000003E4       FindFirstChangeNotification
 0001:000003EC       FindFirstFile
 0001:000003F4       FindNextChangeNotification
 0001:000003FC       GetCurrentDirectory
 0001:00000404       GetLastError
 0001:0000040C       InitializeCriticalSection
 0001:00000414       LeaveCriticalSection
 0001:0000041C       ReleaseMutex
 0001:00000424       SetCurrentDirectory
 0001:0000042C       SetErrorMode
 0001:00000434       WaitForMultipleObjects
 0001:0000043C       WaitForSingleObject
 0001:00000444       lstrlen
 0001:0000044C       ClientToScreen
 0001:00000454       CreatePopupMenu
 0001:0000045C       DestroyMenu
 0001:00000464       SendMessage
 0001:0000046C       TrackPopupMenu
 0001:00000474       CopyMemory
 0001:0000047C       Finalization
 0001:000004AC       Windows
 0001:000004C4       Finalization
 0001:000004F4       Messages
 0001:000009DC       ImageList_GetIconSize
 0001:000009E4       ListView_RedrawItems
 0001:00000A00       ListView_EditLabel
 0001:00000A18       Finalization
 0001:00000A48       CommCtrl
 0001:00000A88       Finalization
 0001:00000AB8       Imm
 0001:0000100C       SHGetDesktopFolder
 0001:00001014       SHGetMalloc
 0001:0000101C       SHGetSpecialFolderLocation
 0001:00001024       Finalization
 0001:00001054       ShlObj
 0001:0000105C       Finalization
 0001:0000108C       UrlMon
 0001:00001094       Finalization
 0001:000010C4       WinInet
 0001:000010CC       Finalization
 0001:000010FC       RegStr
 0001:00001104       SHGetFileInfo
 0001:0000110C       ShellExecute
 0001:00001114       ShellExecuteEx
 0001:0000111C       Finalization
 0001:0000114C       ShellAPI
 0001:0000125C       Finalization
 0001:0000128C       WinSpool
 0001:00001294       Finalization
 0001:000012C4       CommDlg
 0001:000012CC       Finalization
 0001:000012FC       Dlgs
 0001:00001344       Finalization
 0001:00001374       RichEdit
 0001:00001434       Finalization
 0001:00001464       ShellConsts
 0001:0000402C       CreatePIDL
 0001:00004090       NextPIDL
 0001:0000409C       StripLastID
 0001:000040BC       GetItemCount
 0001:000040D4       GetPIDLSize
 0001:000040F8       CopyPIDL
 0001:00004124       ConcatPIDLs
 0001:00004180       DisposePIDL
 0001:000041D0       RelativeFromAbsolute
 0001:000041F8       CreatePIDLList
 0001:00004234       DestroyPIDLList
 0001:00004268       NoFolderDetails
 0001:000042F4       DesktopShellFolder
 0001:00004304       CreateDesktopFolder
 0001:00004380       SamePIDL
 0001:000043DC       DesktopPIDL
 0001:000043F8       GetCSIDLType
 0001:0000440C       IsElement
 0001:00004414       GetShellImage
 0001:00004454       GetCaps
 0001:0000454C       GetProperties
 0001:00004670       GetIsFolder
 0001:000046D8       GetHasSubFolders
 0001:00004740       GetHasSubItems
 0001:00004810       StrRetToString
 0001:00004928       GetDisplayName
 0001:00004A10       ObjectFlags
 0001:00004A38       InvokeContextMenu
 0001:00004C9C       DoContextMenuVerb
 0001:00004D58       GetIShellFolder
 0001:00004E28       GetIShellDetails
 0001:00004EF8       GetIShellFolder2
 0001:00004FC8       CreateRootFromPIDL
 0001:00005050       CreateRootFolder
 0001:000051C4       TShellFolder.Create
 0001:00005330       TShellFolder.Destroy
 0001:00005380       TShellFolder.GetDetailInterface
 0001:00005468       TShellFolder.GetShellDetails
 0001:000054C0       TShellFolder.GetShellFolder2
 0001:00005518       GetDetailsOf
 0001:000055DC       CalcFileSize
 0001:00005634       CalcModifiedDate
 0001:000056A0       DefaultDetailColumn
 0001:00005774       AddDetail
 0001:00005810       TShellFolder.LoadColumnDetails
 0001:0000599C       TShellFolder.GetDetails
 0001:00005A40       TShellFolder.SetDetails
 0001:00005A78       TShellFolder.ParentShellFolder
 0001:00005AA4       TShellFolder.Properties
 0001:00005AF8       TShellFolder.Capabilities
 0001:00005B4C       TShellFolder.SubFolders
 0001:00005B9C       TShellFolder.IsFolder
 0001:00005BEC       TShellFolder.PathName
 0001:00005C40       TShellFolder.DisplayName
 0001:00005CA8       TShellFolder.Rename
 0001:00005DB8       TShellFolder.ImageIndex
 0001:00005DC4       TShellFolder.ExecuteDefault
 0001:00005E10       NotifyOptionFlags
 0001:00005E64       TCustomShellChangeNotifier.Change
 0001:00005EA0       TCustomShellChangeNotifier.Create
 0001:00005F08       TCustomShellChangeNotifier.Destroy
 0001:00005F50       TCustomShellChangeNotifier.SetRoot
 0001:00005F78       TCustomShellChangeNotifier.SetFilters
 0001:00005F8C       TCustomShellChangeNotifier.SetOnChange
 0001:00005FBC       TCustomShellChangeNotifier.SetWatchSubTree
 0001:00005FC8       NotifyOptionFlags
 0001:0000601C       TCustomShellChangeNotifier.Start
 0001:00006080       TShellChangeThread.Create
 0001:000060EC       TShellChangeThread.Destroy
 0001:00006128       TShellChangeThread.Execute
 0001:000061F0       TShellChangeThread.SetDirectoryOptions
 0001:0000626C       TCustomShellTreeView.Create
 0001:0000637C       TCustomShellTreeView.ClearItems
 0001:00006428       TCustomShellTreeView.CreateWnd
 0001:00006470       TCustomShellTreeView.DestroyWnd
 0001:00006484       TCustomShellTreeView.CommandCompleted
 0001:000065C0       TCustomShellTreeView.ExecuteCommand
 0001:00006708       TreeSortFunc
 0001:00006770       TCustomShellTreeView.InitNode
 0001:000068E0       TCustomShellTreeView.PopulateNode
 0001:00006A58       TCustomShellTreeView.SetObjectTypes
 0001:00006A6C       TCustomShellTreeView.CreateRoot
 0001:00006C7C       TCustomShellTreeView.CanExpand
 0001:00006D9C       TCustomShellTreeView.Edit
 0001:00006E4C       TCustomShellTreeView.MouseUp
 0001:00006E68       TCustomShellTreeView.NodeFromRelativeID
 0001:00006EAC       TCustomShellTreeView.NodeFromAbsoluteID
 0001:00006F1C       TCustomShellTreeView.Delete
 0001:00006F48       TCustomShellTreeView.RootChanged
 0001:00006FD4       TCustomShellTreeView.FolderExists
 0001:00007068       TCustomShellTreeView.RefreshEvent
 0001:00007088       TCustomShellTreeView.Refresh
 0001:00007384       TCustomShellTreeView.Notification
 0001:000073C4       TCustomShellTreeView.CanChange
 0001:000074DC       TCustomShellTreeView.GetFolder
 0001:000074F8       TCustomShellTreeView.SelectedFolder
 0001:00007518       TCustomShellTreeView.GetPath
 0001:00007544       TCustomShellTreeView.SetPath
 0001:00007640       TCustomShellTreeView.SetPathFromID
 0001:000077C0       TCustomShellTreeView.SetRoot
 0001:00007800       TCustomShellTreeView.GetImageIndex
 0001:00007810       TCustomShellTreeView.GetSelectedIndex
 0001:00007820       TCustomShellTreeView.WndProc
 0001:00007920       TCustomShellTreeView.SetUseShellImages
 0001:00007968       TCustomShellTreeView.WMDestroy
 0001:00007970       TCustomShellTreeView.Loaded
 0001:00007984       TCustomShellTreeView.DoContextPopup
 0001:000079D4       TCustomShellTreeView.SetComboBox
 0001:00007A24       TCustomShellTreeView.SetListView
 0001:00007A74       TCustomShellTreeView.SetAutoRefresh
 0001:00007B80       TCustomShellComboBox.Create
 0001:00007C54       TCustomShellComboBox.ClearItems
 0001:00007D00       TCustomShellComboBox.CreateRoot
 0001:00007E3C       TCustomShellComboBox.CreateWnd
 0001:00007E90       TCustomShellComboBox.DestroyWnd
 0001:00007EA4       TCustomShellComboBox.SetObjectTypes
 0001:00007EB8       TCustomShellComboBox.TreeUpdate
 0001:00007F44       TCustomShellComboBox.SetTreeView
 0001:00007F94       TCustomShellComboBox.SetListView
 0001:00007FE4       TCustomShellComboBox.Notification
 0001:00008038       TCustomShellComboBox.GetFolder
 0001:00008070       TCustomShellComboBox.InitItem
 0001:000080D4       ListSortFunc
 0001:00008188       ComboSortFunc
 0001:000081B4       TCustomShellComboBox.AddItems
 0001:000083D0       TCustomShellComboBox.Init
 0001:00008490       TCustomShellComboBox.IndexFromID
 0001:0000850C       TCustomShellComboBox.SetRoot
 0001:0000854C       TCustomShellComboBox.RootChanged
 0001:000085D4       TCustomShellComboBox.GetPath
 0001:0000861C       TCustomShellComboBox.SetPath
 0001:00008718       InsertItemObject
 0001:000087B0       TCustomShellComboBox.SetPathFromID
 0001:00008968       TCustomShellComboBox.GetShellImageIndex
 0001:00008984       TCustomShellComboBox.SetUseShellImages
 0001:00008A34       TCustomShellComboBox.Destroy
 0001:00008A68       TCustomShellComboBox.Loaded
 0001:00008A7C       TCustomShellComboBox.Change
 0001:00008B50       TCustomShellComboBox.Click
 0001:00008BF4       TCustomShellListView.Create
 0001:00008D10       TCustomShellListView.Destroy
 0001:00008D48       TCustomShellListView.ClearItems
 0001:00008DA0       TCustomShellListView.CommandCompleted
 0001:00008E68       TCustomShellListView.ExecuteCommand
 0001:00008FB0       TCustomShellListView.CreateWnd
 0001:00009020       TCustomShellListView.DestroyWnd
 0001:00009034       TCustomShellListView.SetObjectTypes
 0001:00009050       TCustomShellListView.RootChanged
 0001:000090E4       TCustomShellListView.Populate
 0001:00009338       TCustomShellListView.Notification
 0001:00009378       TCustomShellListView.DblClick
 0001:00009448       TCustomShellListView.EditText
 0001:00009474       TCustomShellListView.Edit
 0001:00009514       TCustomShellListView.SetAutoRefresh
 0001:000095F4       TCustomShellListView.SetRoot
 0001:00009644       TCustomShellListView.SelectedFolder
 0001:00009674       TCustomShellListView.OwnerDataFetch
 0001:000097B0       TCustomShellListView.GetFolder
 0001:000097C8       TCustomShellListView.OwnerDataFind
 0001:00009898       TCustomShellListView.SetSorted
 0001:000098B8       TCustomShellListView.Loaded
 0001:000098E8       TCustomShellListView.DoContextPopup
 0001:0000993C       TCustomShellListView.Back
 0001:00009998       ColumnIsUnique
 0001:00009A24       AddColumn
 0001:00009B3C       AddDefaultColumn
 0001:00009BA4       AddDefaultColumns
 0001:00009C7C       TCustomShellListView.EnumColumns
 0001:00009E8C       TCustomShellListView.KeyDown
 0001:00009F40       TCustomShellListView.SetViewStyle
 0001:00009F64       TCustomShellListView.SetTreeView
 0001:00009FB4       TCustomShellListView.SetComboBox
 0001:0000A004       TCustomShellListView.TreeUpdate
 0001:0000A03C       TCustomShellListView.WndProc
 0001:0000A08C       TCustomShellListView.Refresh
 0001:0000A154       TCustomShellListView.SetPathFromID
 0001:0000A1A8       TCustomShellListView.CreateRoot
 0001:0000A1CC       TCustomShellListView.SynchPaths
 0001:0000A284       Finalization
 0001:0000A2EC       ShellCtrls
 0001:0000A504       @GetPackageInfoTable
 0001:0000A50C       @PackageLoad
 0001:0000A518       @PackageUnload
 0001:0000A524       vclshlctrls
 0002:00000000       TlsIndex
 0002:00000004       Module
 0002:0000001C       TlsProc
 0002:0000002C       IID_IContextMenu
 0002:0000003C       IID_IShellFolder
 0002:0000004C       IID_IContextMenu2
 0002:0000005C       IID_IShellFolder2
 0002:0000006C       IID_IShellDetails
 0002:0000007C       nFolder
 0002:000000D8       cmvProperties
 0002:000000DC       ICM
 0002:000000E0       ICM2
 0002:000000E4       DesktopFolder
 0002:000000E8       CompareFolder
 0002:000000EC       R
 0002:00001000       ModuleIsLib
 0002:00001001       ModuleIsPackage
 0002:00001004       HInstance
 0002:00001008       .1
 0002:0000100C       tlsBuffer
 0002:00001010       .3
 0002:00001014       .1
 0002:00001018       .1
 0002:0000101C       .1
 0002:00001020       .1
 0002:00001024       .1
 0002:00001028       .1
 0002:0000102C       .1
 0002:00001030       .1
 0002:00001034       .3
 0002:00001038       .1
 0002:0000103C       .1
 0002:00001040       .1
 0002:00001044       .1
 0002:00001048       .21
 0002:0000104C       CS


Line numbers for vclshlctrls(vclshlctrls.dpk) segment .text

    38 0001:0000A524

Bound resource files

vclshlctrls.res
C:\DOCUME~1\~KOKOP~1\LOCALS~1\Temp\dtf2956.tmp


Program entry point at 0001:0000A524
